:020000040000FA
:100000000128831203138501831606309F00CF3029
:10001000850007309C00831600308500860083121F
:10002000C001850186018B204E207320442076205C
:1000300044201928820746346F347234743479347A
:100040002034583432342034643469347334703496
:100050006C346134793420346434723469347634E5
:10006000653472342E34543465347334743420342B
:1000700062347934203444346134763465342E3437
:100080005334313430340034C00140081A20003A6F
:1000900003194D286620C00A452800342030592015
:1000A00028305920063059200C30592085209520C1
:1000B0000034C400440E0F3986008510A420440883
:1000C0000F3986008510A42093200034C400440E0C
:1000D0000F3986008514A42044080F398600851442
:1000E000A42095200034803059200034C03059209D
:1000F0000034803E59200034C03E592000340D3079
:10010000592000340C30592000340130592000347B
:100110002E306620080064309828503098283230FD
:100120009828143098280A309828053098280130EB
:10013000C100C730C2000530C300C20BA028C30BEA
:100140009D28C10B992800340515000005110034C5
:02400E00723FFF
:00000001FF
